:030000000219FDE5
:03000B000200AA46
:03002B000201656A
:03005B000202FBA3
:030073000202E1A5
:1000800002030406080C10182030406080040608A3
:100090000C10182030406080A0C000070F1F3F0DDB
:1000A0000D0403060D0503030202C2AFC0D0C0E079
:1000B000206217E5256002E473E525F4F58A758B67
:1000C00000D262D0E0D0D0D2AF3285268AC262E5BB
:1000D00026F46035306803207210758B00D0E0D0B4
:1000E000D0D292D291D290D2AF32D292D291D2903B
:1000F000206E0C206609740AD5E0FDE57E429075FD
:100100008B00D0E0D0D0D2AF32758A00C28DD262DF
:1001100001FF01B9306805206602C29201B930685A
:1001200005206602C29101B9306805206602C290BE
:1001300001B9C29330680A2066077408D5E0FDC291
:100140009201B9C29430680A2066077408D5E0FDB0
:10015000C29101B9C29530680A2066077408D5E0DB
:10016000FDC29001B9C2AFC2AD53E6EFC0D0C0E04E
:10017000D2D3D2AFC2CEE52A6007207449152A2116
:10018000C67800790020742EE580307E01F430E4DA
:100190000278FF53DACF207E0343DA20307E034318
:1001A000DA10C2D8C271E580307E01F430E4027901
:1001B000FFC3E89970CB306103752A402074037542
:1001C0002A40885FD27020740DE52B6004152B2126
:1001D000D643DA01C2D820700221E9A85F2061026B
:1001E000C27020740221E788227882B60403852237
:1001F00024C3E52594404002D26420CF0AD0E0D049
:10020000D043E610D2AD32C2CF053A7802E52A607B
:1002100005307402152AC3E55F940140057562003C
:100220004133756300756C00E5622401F56250038B
:100230007562FF7982B7020D306D1DC3E5229432DD
:100240004016854D227982B7030E306D0BC3E5222F
:1002500094324004798E8722C3E5239522600840BA
:1002600004152341670523D8CA056CE56C70021597
:100270006CD56D63756D017805C3E56C956E40575F
:10028000C3E56C956F50087801756D0302029BC33E
:10029000E56C957050057801756D01C3E565952491
:1002A000401E7982B7040241CC206D14852465E597
:1002B0006C046003856E6C756D0175233C0202D77A
:1002C000E5652850057565FF41CCF565E565047069
:1002D000067563FF756CFFD0E0D0D043E610D2AD59
:1002E00032C2AFC0D053E67FC2607591008556948C
:1002F000855795759104D0D0D2AF32C2AF53E6EF97
:10030000C2ADC0D0C0E0C0F0D2D3D2AFA8FBA9FC30
:10031000C2D8307102616253DACF207E0343DA1013
:10032000307E0343DA20D271E580307E01F420E490
:1003300002613988278928A14753DACF207E0343F9
:10034000DA20307E0343DA10C2D8C271307402A1C1
:10035000337800E580307E01F430E402A133885F19
:10036000A11B53DACF207E0343DA20307E0343DA29
:1003700010C271206102813B53DACF207E0343DA41
:1003800010307E0343DA20C2D8D271885A895BC309
:10039000E89558F8E99559F97B007E087A00C3E89A
:1003A000948CE994005005755E00812D882178A217
:1003B000E6A8216055C3E894C8E994005008E4D247
:1003C000E4FB7A0A8108C3E89468E994015008E4E0
:1003D000D2E3FB7A0F8108C3E894D0E99402500875
:1003E000E4D2E2FB7A1E8108C3E894A0E9940550A8
:1003F00008E4D2E1FB7A3C8108C3E89498E99408C8
:100400005008E4D2E0FB7A787E00C3E8955CFCE912
:10041000955DFD30E70AECF42401FCEDF43400FDB9
:10042000755E00C3EC9AED9E5003755E01885C8991
:100430005D855A58855B597802A11BC3E89527F85A
:10044000E99528F9307C0281FF307B0281FF307A08
:100450000281F8207502815EE9FDE8FC817DE9C337
:1004600013F9E813F830790281F8E9C313F9E813B6
:0D047000F830780281F8E9C313FDE813FCB1
:10047D0020612CC3EC941CED940240028194ED702C
:10048D001EC3EC94C850180529E52970021529C31F
:10049D00E529940A5002A133755F00D270A133E5AE
:1004AD0029600215297400207F037896E624FAFE50
:1004BD00E43400FFC3EC9EFCED9FFD5006780079FF
:1004CD000081FFC3EC94FFED9400400678FF7900A6
:1004DD0081FFEC8575F0A4C5F0A2F733F8790040E3
:1004ED000302051B78FF790002051BE9C313F9E828
:1004FD0013F8307C0EE9600278FFC3E81338F8E496
:10050D003400F9C3E894FFE99400400278FF885F56
:10051D00D270206102A133741FF4552F4BF52FC2F9
:10052D0074EB7002D274752A40307403752A0A3048
:10053D006102A14720740353DAFE207403752B204A
:10054D00D0F0D0E0D0D0D2AD43E610327901020523
:10055D00777903020577790A020577791E02057707
:10056D00796402057779C80205777817E4D5E0FD3F
:10057D00D8FAD9F6227A147B7802059E7A107B8CF4
:10058D0002059E7A0D7BB402059E7A0B7BC802058F
:10059D009E7902B27DE4C294D5E0FDC291D5E0FD15
:1005AD00D291D5E0FDD294D5E0FDC292E576D5E0AD
:1005BD00FDD2927496D5E0FDD9D9EAF8D5E0FDD8F3
:1005CD00FBDBCEC29422C37C007D0075F00005F0EC
:1005DD00EA33FAEB33FB50F6EB13FBEA13FAC3E9FC
:1005ED00FFE8FEE89AF8E99BF95004EFF9EEF8B34D
:1005FD00EC33FCED33FDD5F0DFEDF9ECF822E889B5
:10060D00F08A20D2D4F8A9F07B0030F70B7BFFF4F1
:10061D002401F8E9F43400F9E88520F0A4ADF0F8F0
:10062D00E98520F0A4AFF0FEED2EF974003FFA7CC1
:10063D0004C3EA13FAE913F9E813F8DCF48BF0308C
:10064D00F70AE8F42401F8E9F43400F9E889F0C276
:10065D00D4F8A9F0227882B60403020701C3E55F3E
:10066D009419401EE52D54067018206D36780579C5
:10067D0094E7146007780A1460027812C3E5419874
:10068D00401F306D09856765756CFF756D0185229D
:10069D0024E4F545F546F547F548F549C26D0207E1
:1006AD0001D26D7994E7147013E523F43333F91304
:1006BD00F8E9540104F9E854FE0206F5E714147044
:1006CD0014E523F4333333F913F8E9540304F9E84B
:1006DD0054FC0206FDE523F433333333F913F8E903
:1006ED0054070404F9E854F8C39440F8E99400F968
:1006FD008845894622C3E54113F9E54013F8C3E562
:10070D004598F8E54699F9500CC3E89480E994FFB3
:10071D004016020739C3E8947FE99400500302079D
:10072D0039787F7900020739788079FF884A894BBB
:10073D0022E54A2547F8E54B3548F9854B20E4304D
:10074D000701F43549FA30E709C3EA94F040150280
:10075D000777C3EA940F500302077778FF79FF7A82
:10076D000F020777780079007AF0C3E5249564507D
:10077D000AC374019524500B020795E54B20E70E33
:10078D00020795E54B30E706884789488A49227864
:10079D00A4E6FAC3E54A33F8E54B33F9D10BE9305A
:1007AD00E70BC3E89480E994FF4013E1CFC3E894CD
:1007BD007FE994005002E1CF787F7900E1CF788016
:1007CD0079FFE820E715C3E52398F84009C3E894BD
:1007DD000140030207F678010207F6E8F42401252B
:1007ED0023F840030207F678FF884C2278A5E6FA35
:1007FD00A848A94912060BE930E70CC3E89401E9B2
:10080D0094FF401602082BC3E894FFE994005003AF
:10081D0002082B78FF790002082B780179FFE92077
:10082D00E715C3E54C98F84009C3E894014003026D
:10083D0008527801020852E8F42401254CF84003CF
:10084D0002085278FF88242278FFC26420693D2077
:10085D006A12D264C3E541940A4009C3E525944068
:0F086D005002C26479A1E76023E541601F74FF68
:10087C008541F0848539F0306A0375F005A4F8C51C
:10088C00F0600278FFC3E895675002A8678866227B
:10089C00C3E5409440E5419401E56650031401AD75
:1008AC00046002F566227883E6F520120F5475E891
:1008BC009012055975E890E5E820ECFBA8BDA9BE9F
:1008CC00120FF27571AF757200C3740013FD74AF23
:1008DC00606613FC74AF2CFC74003DFDECFAEDFB70
:1008EC00C3E89AE99B4014E57124AFF571E57234C5
:1008FC0000F572EA2CFAEB3DFB80E5AE71AF72C3EA
:10090C00E57213F9E57113F8C3E913F9E813F87AF2
:10091C0003C3E913F9E813F8DAF7AA201A7009757A
:10092C0071007572000209441AEA6008EE28FEEFA5
:10093C0039FFDAF88E718F722275E890227883E68F
:10094C00FFE5E820ECF7A8BDA9BE0573C3E57394D9
:10095C00084052757300E9FA79A0E76044EA700721
:10096C00E574601B02097FC3E895746010E5745050
:10097C0006600C1402098B0460F902098BE574F50E
:10098C0074C39458401B7564C0C3940440137564BD
:10099C0080C39404400B756440C394044003756495
:1009AC000075BB0322EFC39401601F74AF601BC3BF
:1009BC00E894FFE994035012C3E89571E9957250DD
:1009CC0009E564600C15640209DDE564F460020558
:1009DC0064A864C3E524985002A824C3E895654034
:1009EC000AA865E565F4600385656488258826E5B5
:1009FC0073B4070375BB1022743279A687F0A4C5B3
:100A0C00F0A2F733F8C3E895644002A86488228802
:100A1C0024882588268867227540007541F022C2FB
:100A2C00AF75C820A8CCA9CDAA3A30CF010A75C899
:100A3C0024D2AFAB3BAC3C883B893CC3E89BF8E988
:100A4C009C206908F93067026140419DAD3D8A3DAB
:100A5C00F9EA9DFA600478FF79FFAE3EAF3F8B3E1A
:100A6C008C3FC3EC9FFCC3E99CF542A83BA93CC35B
:100A7C00E89EF8E99FF9C3E54113FBE54013FAE85A
:100A8C002AF540E93BF54150067540FF7541FF41A1
:100A9C00E7AA40AB41AC40AD417E047F02C3EB946E
:100AAC000440021E1FC3EB940840021E1FC3ED132B
:100ABC00FDEC13FCDEF7C3EA9CFAEB9DFBEF60093F
:100ACC00C3E913F9E813F8DFF7EA28FAEB39FB8AE4
:100ADC00408B4150067BFF8B408B41C3EB94025003
:100AEC0002D2673069047F0361127892E6FFC3E596
:100AFC0037948240110FC3E53794A040010FC3EF28
:100B0C00940640027F057E05E541C4540FF9E5418A
:100B1C00C454F0F8E540C4540F28F8C3E89EFAE931
:100B2C009400FB4009C3EA9402EB940050047A024F
:100B3C00E4FB618CAA40AB41EBC4FEEAC4540F4EFB
:100B4C00FCC3EA9CFAEB9400FBC3E813C313F8EA6A
:100B5C0028FAEB3400FB8A408B41C3EB9402400231
:100B6C00C2677805EBC4FE7B00EAC4540F4EFAC38F
:100B7C00EA98FA4005C3940250027A027892E6FF92
:100B8C00306002618C855256855357D26043E680A3
:100B9C00C3E49AF8E49BF93067028126E8FAE9FB92
:100BAC00D3E913FDE813FC88528953C3EF94036017
:100BBC0038EF20E00DE82CF8E93DF9ECFAEDFB02FA
:100BCC000BE1E828F8E939F9C3E82402F8E9340024
:100BDC00F97AFE7BFFC3EF9403400E8A548B558841
:100BEC004E894F8C508D51815A885489558A4E8B21
:100BFC004F8C508D51306920C3E53394034019E577
:100C0C0042A2E713F8E555F4240138400B20E7081D
:100C1C007554FFF42401F555815AE8FAD3E813FC16
:100C2C008852C3EF94036020EF20E007E82CF8EC27
:100C3C00FA8146E8282402F87AFEC3EF94034008B0
:100C4C008A54884E8C50815A88548A4E8C50E56B4D
:100C5C00C3335002646BF56B3060028164753402EF
:0F0C6C00D26043E680E52D54066026A840A941DA
:100C7B00C3E913F9E813F8C2AF53E67F759100C3CC
:100C8B00E498F594E499F595759104D26043E68068
:100C9B00D2AF22D265754400752000306B037520EE
:100CAB0040020CBDD265754400752040306B037556
:100CBB002000D2AF7801206722E52D54066002C2D6
:100CCB0065C3E54194054013780294054008780309
:100CDB00940540027806306902780A206019E544D1
:100CEB00601530690AC3E53394034003D53406D24B
:100CFB00AFD26CA18F916CD2AF0000C2AF20672630
:100D0B00E541C3FB940F40027B0FEB2405307301CD
:100D1B0023306A02742820620123F9306902798238
:100D2B00E58BC39940B50544E59BF45440B52002CF
:100D3B00A17930690A08C3E8940A40010881E620CA
:100D4B00650281BDC26553E67F75910030671075F2
:100D5B0094007595FE759104D26043E68081BDAE1B
:100D6B0040AF41C3E49EF594E49FF595A160C3E5C4
:100D7B00339402500281BD30650281BDD802A18D32
:100D8B0081E6C26C53E67F75910085549485559529
:100D9B00759104854E56854F57D26043E680D2AF8E
:100DAB00E52D54066008206A020533020DC9306C2C
:100DBB000D206B0A2065071581158102162F2278ED
:100DCB00003064053065027801E53775F007A4F94A
:100DDB00E5F028F5F0E9A2F013A2F113A2F213F556
:100DEB0037C394785003753778C3E5379538400887
:100DFB00D266D292D291D290306002C10385505606
:100E0B00855157D26043E68022D2A0207D11C2AF1C
:100E1B00754302C294D293D2AF759F10020FEFC2EB
:100E2B00AF754302C294D295D2AF759F10020FEFEC
:100E3B00C2A0307243207D20C2AF754303900143A3
:100E4B00757E10D290C295306204C291C15BD29470
:100E5B00D2AF759F20020FEFC2AF754303900143D2
:100E6B00757E10D292C293306204C291C17BD29430
:100E7B00D2AF759F00020FEF207D17C2AF754303F2
:100E8B0090011ED290306202C291D2AF759F2002A8
:100E9B000FEFC2AF75430390011ED292306202C2B4
:100EAB0091D2AF759F00020FEFD2A0207D11C2AF80
:100EBB00754304C293D295D2AF759F00020FEFC258
:100ECB00AF754304C295D293D2AF759F20020FEF3B
:100EDB00C2A0307243207D20C2AF75430590013212
:100EEB00757E08D291C294306204C292C1FBD29338
:100EFB00D2AF759F10020FEFC2AF7543059001542F
:100F0B00757E20D291C294306204C290E11BD295BF
:100F1B00D2AF759F10020FEF207D17C2AF7543053F
:100F2B00900114D291306202C292D2AF759F10021F
:100F3B000FEFC2AF754305900128D2913062EBC21F
:100F4B0090D2AF759F10020FEFD2A0207D11C2AFD0
:100F5B00754306C295D294D2AF759F20020FEFC294
:100F6B00AF754306C293D294D2AF759F00020FEFB9
:100F7B00C2A0307242207D20C2AF75430190015454
:100F8B00757E20D292C293306204C290E19BD295BF
:100F9B00D2AF759F00020FEFC2AF754301900132C4
:100FAB00757E08D290C295306204C292E1BBD29397
:100FBB00D2AF759F20E1EF207D16C2AF7543019034
:100FCB000128D292306202C290D2AF759F00E1EF3E
:100FDB00C2AF754301900114D290306202C292D21B
:100FEB00AF759F20C26622900112757E00D292D2FD
:100FFB0091D290C293C294C295C262227880760736
:10100B000876070876010876040876FF0876FF084D
:10101B00760A087602087601087601788C76010844
:10102B0076000876B40876FF0876FF0876FF087618
:10103B00030876FF0876010876FF0876250876D038
:10104B000876780876C80876040876FF08760108D3
:10105B00760008767A08760A087601087601087613
:0E106B00000876FF227887E6FFC272BF0302FC
:10107900D2727888C27DE630E102D27DC27E78895B
:10108900E630E102D27EC3EF94026008758E01D288
:10109900730210A2758E00C273227880E614900044
:1010A900809378A4F67881E6149000809378A5F669
:1010B9007886E61490008D9378A6F6789FE6F87006
:1010C9000108C3E8941140027811E82828F56E2533
:1010D9006E256E28F56F256E2828F570789CE675C3
:1010E90038FF75390CB402067538A075390AB4038E
:1010F9000675388275390578A3E61490009A93F538
:1011090069120FF222227896E6FA7897E6FB788838
:10111900E6B40305C3EB940EFB307F047A007BFF32
:10112900C3EB9AFCC3948250027C827575000575E5
:10113900EC8575F0A4C3E5F0947D40F222D27F31AD
:101149000F1205687A007B007C1012055EE55F2AA4
:10115900FA74003BFBDCF37C04C3EB13FBEA13FAE0
:10116900DCF7FEC27F310F22E5EF20E60375200090
:101179000520903FFFE520146006901DFF146000D4
:101189009304600375EF1253D9BF7581C043FF8083
:1011990012055975EF0243B203E5B3240420E70DA4
:1011A900F521E5E320E0068521B343E301120FF2BF
:1011B9007580FF75A40075F1D475D4EF75908775A6
:1011C900A54075F2FF75D5BF75A60175E24275DBBD
:1011D9004675EA02E4F8F6D8FD756B011107121697
:1011E9007778988676753001C2AF1205721205823A
:1011F9001205681205891205681205901205681210
:10120900179912057212057212056DC2AF78FA7933
:10121900FA308407D9FBD8F7021C00117011A331E9
:101229000E310F78988676120FF2758850758912EB
:1012390075C82475910475D84075A82275B80275CA
:10124900E690759B80759D0075D10E75BC5875BB70
:101259000375BA1175E880120559D2AF1208B25355
:10126900DACF207E0343DA20307E0343DA1043DAF3
:1012790001C2D8C271120572D2617B037A0CE55E94
:1012890070077A0CDB03021214120568207003023E
:101299001214C270E55FC3940240E1E52F541F8523
:1012A9006160F561B560D5DAD5C26153DACF207EC8
:1012B9000343DA20307E0343DA10C2D8C27178A220
:1012C900E67008D274E52F54E0F52FC27575290030
:1012D90012056D307409C3E529940A4002D27512CA
:1012E900055E78023074027800C3E55F9840F0C269
:1012F900AF120582120582120582D2AF12057275EC
:101309004D0012055E788CE6C3940150030213E187
:10131900E530C3940150030213E1207435C3E55F3E
:1013290094FF50030213E1C2AF120597D2AF120521
:101339006DC3E55F940150EFC2AF120582120563D8
:10134900120582D2AF12056DC3E55F94FF40E90231
:10135900181E7F05D27F310F12056DC2AFC27F31D2
:101369000FAE5FC3E55F947FD2AF4076120559C2D5
:10137900AF120597D2AFDFDC3146C3EE94057897FB
:10138900F61205721216B81217A17F0AD27F310F11
:1013990012056DC2AFC27F310FAE5FC3E55F947FA7
:1013A900D2AF50E6120559C2AF1205821205631277
:1013B9000582D2AFDFD63146EE24057896F61205BE
:1013C900721216B81217D012056D310FC3E55F946A
:1013D900FF5002612302181EC3E55F954D40038546
:1013E9005F4D12056D78017988E7B403027805C36A
:1013F900E55F984002610BC2AF120597120597127B
:101409000597D2AF120572753000E4F531F5320552
:1014190031E531F470390532789AE6781914601299
:10142900783214600D787D14600878FA14600375B9
:101439003200C3E53298401715327531B478998670
:1014490076C2AF120597D2AF7898867612056D12DB
:101459000563E52A7005307402411478012074028D
:0F1469007806C3E55F9840A712056DE52A70036A
:10147800021214C2AF120FF2E4F522F523F524F597
:1014880025F526F56AD2AF7885E6C333F568E4F525
:1014980045F546F547F548F549F573F52CF52DF56D
:1014A8003775730875BB10120559120945E5E82010
:1014B800ECFBA8BDA9BEE97001F88874120949754A
:1014C800730875BB107887E6FE760211707887EE90
:1014D800F6C2AF7564FF120A048522648522658509
:1014E8002266D2AF75220175240175250175260182
:1014F80085636C756D017888E6B40307C27D307624
:1015080002D27DD268D269753300120F54120F7B54
:10151800120A24120A2B120A24120A2B120A240273
:101528001536C2AF1170D2AF75730075BB03120CBC
:10153800AF120662120DCA120E14120A2B120C9E5A
:10154800306D031207022067031208553067031233
:10155800089C120DCA120E3B120A2B120CAF306DEA
:101568000312073E120DCA120EB4120A2B120C9E59
:10157800306D0312079C120DCA120EDB120A2B12D1
:101588000CAF306D031207F9120DCA120F54120A6C
:101598002B120945120C9E120DCA120F7B12094913
:1015A800120A2B30692F206B2C8567648567658547
:1015B800636C756D0179187A0CC3E533994009C2DB
:1015C80069D26A8A350215DDC3E55F9401400302DA
:1015D8001536021637306A1B206B18E5351470046F
:1015E800C26AA12AF535C3E55F94014003021536A6
:1015F800021637753600C3E56294014009856765B0
:1016080085636C756D01C3E56278FA985021307472
:1016180004E52A601A78F0306B058567647820C382
:10162800E541985002A1360536E55F6002C13A757A
:101638003600C2AF120FF27887E6FE760211707894
:1016480087EEF6E4F522F523F524F525F526F56869
:10165800C268D2AF120559120FF2307406E52A702B
:10166800024114788DE6C39401400241E881139049
:101678001A0D78201216FAE520B4A50CA31216FA52
:10168800E520B45A0302169811071216B80216B7C5
:10169800901A0378807B0A1216FAA308DBF9901ACD
:1016A8000F788C7B181216FAA308DBF9901A2722F8
:1016B800C2AF121739121713901A00740E1216FFC0
:1016C800A374041216FFA374141216FF901A037859
:1016D800807B0A1216FEA308DBF9901A0F788C7B20
:1016E800181216FEA308DBF912174C12172A901AC3
:1016F8002722E493F622E6438F01538FFD75EF020C
:1017080075B7A575B7F1F0538FFE22438F02438F4B
:101718000175EF0275B7A575B7F1901A0DF0538FE3
:10172800FC22901A0D74A5D1FF901A0E745AD1FF9D
:10173800227A3079D07820901A40D1FAE520F7093A
:10174800A3DAF7227A3079D0901A40E7D1FF09A3BB
:10175800DAF922AB77A878BB01027980BB0202795B
:1017680081BB03027982BB04027994BB05027983A9
:10177800BB06027986BB07027992BB08027987BB50
:101788000902799CBB0A027988BB0B027989E8F7C0
:10179800227C05120572DCFB22C2AF1205821205FB
:1017A80089120590120597120563120582120589A0
:1017B8001205901205971205631205821205891207
:1017C8000590120597D2AF22C2AF12059712059065
:1017D80012058912058212056312059712059012E7
:1017E80005891205821205631205971205901205E4
:1017F80089120582D2AF22AE77AF78C2AF120582C6
:10180800120582120582120563DEF212059712058F
:1018180063DFF8D2AF221217A11217991217997520
:1018280077017578017579001217FF7C05AD5F1295
:101838000572C3ED955F70F5C3E55F9401400AC377
:10184800E55F94FF403702186212175B1216B81250
:1018580017A1C2AF75EF12121799DCD10579C3E54C
:0F186800799403500280C11217990578E577141F
:1018770090009F93F808C3E57898500280A8121744
:10188700991217990577C3E577940C500280941243
:0D18970010071216B8C2AF75EF12121799A4
:0319FD0002117163
:101A00000E041407070104FFFF0A020101A55A0191
:101A100000B4FFFFFF03FF01FF25D078C804FF01DA
:081A200000FF0A010100FFFFB5
:101A400023484B696E67323041232020202020201C
:101A500023424C48454C4923463333302320202031
:101A60002020202020202020202020202020202076
:101C0000C2AFC2D353D9BF7581C043B20343FF8073
:101C1000752438752503B1C975EF0275E24043F1AB
:101C20001053A4EF75D400D2847DFA780379E67C52
:101C300010752200752300901DD67B0675249875BB
:101C400025013084028142208408D8FBD9F9DCF7D1
:101C500081B4308408D8FBD9F9DCF781B4B189E4C8
:101C600093A3C39A6004DDC381B4DBDBB17B600264
:101C7000812B7B08E493FAA3B15CDBF87A30B15C8A
:101C8000752200752300B17BEAFCEBFDC3ED94FEE9
:101C9000400EB17B8A278B28ED30E0048A828B834B
:101CA000B17B7AC270D8C3ED94FE601350CEBD00F4
:101CB00025EC60097520007521FF0200008100A855
:101CC00027A9280809D804D90281D3B17FEA89AAB3
:101CD000F281C50D81A0C3ED94035049EDA2E092BD
:101CE000007AC5C3E5829400E583941C50902000DF
:101CF00010438F02438F0175B7A575B7F1F030001F
:101D00001FA827A9280809438F01538FFDD804D99C
:101D100002A12089AAE275B7A575B7F1F0A3A10DBC
:101D2000538FFC817C7AC1BD030CE493A3FAB140CC
:101D3000DCF8B138817C817EAA22AB23B15CEBFA5E
:101D4000EA6222752608C3E52313F523E52213F57D
:101D50002250066323A0632201D526EAB1C9B1C986
:101D600075260AEAF4200102D284300102C284B14D
:101D7000C9C3134002C201D526EB22B17FEAFB2082
:101D80008402A17F308402A184752608AE24AF2589
:101D9000C3EF13FFEE13FEB1CDB1C9C3EA13308414
:101DA000024480FA30E703632201C3E52313F523DD
:101DB000E52213F52250066323A0632201D526D91C
:101DC000E52265236523F52222AE24AF250E0FDE22
:101DD000FEDFFCD20122424C48656C693437316326
:041DE000F3300601D5
:00000001FF
